:10000000830100308A004728F60003088301D100ED
:100010008B1A0B1D40280B11FC3083120313810037
:10002000AD0A2D08043A031D3928AD01AE0AA11C02
:100030001D28AF0A031D1D28A117211D2328B00A62
:10004000031D23282214A11E3928C00A0319C10A3E
:1000500003304102E830031940020318A112C20A1A
:100060000319C30A013043022C300319420203185A
:100070002113211F4028051F3F280513402805177D
:100080000313831251088300F60E760E0900233005
:1000900084004F30542020308400233054208301CA
:1000A000F62D04068001840A0406031D512800343D
:1000B00083120313CF00D01B6628501B6E285008F4
:1000C0008A004F08CF0A0319D00A82008313501800
:1000D00083174F08CF0A8400000808003E345134CB
:1000E000493445343E34003442347F3440340034A3
:1000F0004234613451344934463421344134453436
:100100004B3431341834143412347F3410342734DF
:1001100045344534453439343C344A34493449341F
:1001200030340134713409340534033436344934FD
:1001300049344934363406344934493429341E3478
:1001400000340034003400340034083408340834F7
:100150000834083400340034C034C034003400346F
:1001600006340934093406343E34413441344134D0
:1001700022342034543454345434783440343834B1
:10018000043404347C34383444344434443438340F
:100190007C341034103410347C34273448344834E0
:1001A00048343F347C342034103408347C347C347C
:1001B000403440347C34C0343E34413441344134E2
:1001C0003E347C3454345434543424347C34143425
:1001D0001434143408347C345034203400347C34E7
:1001E0007C3454345434543428347F340834143434
:1001F00022344134223449344934493436340134C8
:1002000001347F3401340134383454345434543498
:1002100018347C340834103408347C347C3404348E
:10022000043404347C34043404347C34043404341E
:100230000C345034503450343C340034363436347A
:1002400000340034083400340834003408340034F6
:100250000834143422344134413422341434083400
:100260000034143414341434143414343F3440340B
:10027000403440343F347F3449344934493436348F
:100280007E341134113411347E347C341034103403
:1002900028344434283444345434543428344834CE
:1002A0003434143414347C346C3410347C341034CE
:1002B0006C341F342034403420341F347F344934AC
:1002C0004934493441347F340934193429344634AB
:1002D0007F3440344034403440347F340834083470
:0402E00008347F342B
:100670008A308301C400C40B3B2B08000230830185
:10068000C600C60B412B080012308301C600C60B02
:10069000472B08009E308301C400C40B4D2B08007B
:1006A0008301C8008612861037248614080083014F
:1006B000CB00861686103724861408009630B8249E
:1006C0005A30B8246430B8249630B82C8301C7005F
:1006D000460807394038502347087F398038502B67
:1006E000F0000030711870070310F00D0310F10CCA
:1006F000F10803190800722BFF30B8244B30B824DE
:10070000A030B8247830B824E130B824E630B82CD2
:1007100083012E08C5001930C5072E084502C40004
:10072000C4080319080064008D2BF401F5010310BF
:10073000F30CF20C031CA32B7008F40771080318C8
:10074000710AF5070310F00DF10D72087304031917
:100750000034972B8301C60100306623F830C400B3
:100760000130C500640000305723C4080319C503D5
:10077000C4034508803AF00080307002013003194C
:100780004402031C0800B22BB430B824B430B8249F
:10079000B430B824B430B824B430B824B430B82459
:1007A000B430B824B430B824B430B824B430B82449
:1007B000B430B824B430B824B430B824B430B82C31
:1007C00008308301C400C5016400061183160611B8
:1007D00000000000000006153E23A0100619A0141A
:1007E00044230310C50CA01CF72B8030C5073E2303
:1007F000C40BE42B3E234508080064008312031356
:100800008615861400008611882386152130502312
:10081000C230502307305023133050232030502350
:1008200009305023AA23083050230C305023C6012E
:100830000030662B08308301C400C5016400051236
:100840008316051200000000000005163E2320114B
:10085000051A201544230310C50C201D312C8030AF
:10086000C5073E23C40B1E2C3E2345080800830108
:10087000CC0064000830CD00CE010612CC1F422C03
:100880000614432C061006160310CC0DCD080319D0
:10089000CE03CD034E08803AF00080307002013064
:1008A00003194D02031C08003D2C8301C4000830CD
:1008B000C500A0104418A014831203130611831658
:1008C000061100000000000000008312A01C6B2C29
:1008D000831606156D2C8316061144238316061500
:1008E0003E230310C40CC50B592C3E2B053083014D
:1008F000C60000306623D230B824D730B824D730B1
:10090000B824AA30B8249B30B8243730B8247830C3
:10091000B8244B30B824DC30B8247830B824E13027
:10092000B824E630B8249630B8245A30B82C830165
:10093000C4000830C5002011441820158312031389
:10094000051283160512000000000000000083124B
:10095000201DAD2C83160516AF2C831605124423DB
:10096000831605163E230310C40CC50B9B2C3E2B8F
:100970008301C400C900CA010530C700C8014A0884
:10098000003ED00049086E3E0318D00A5820C5002A
:10099000C6015723C90A0319CA0AC7080319C8039D
:1009A000C7034808803AF000803070020130031914
:1009B00047020318BF2C0030572B023083019F00E1
:1009C00086018501BF3083168500C43086008030E3
:1009D0009F0020308B0083128C0183168C0107301E
:1009E0008100FC30831281008B17A013A113A1108A
:1009F0002110221021112113A112A210C201C30142
:100A00004208C0004308C100AD0108006400831221
:100A10000313A401A30183160516061583120512FC
:100A200006118316051206114A23831605160615AC
:100A30004423A0110619A015831203132012051ACE
:100A400020163823A0120619A016831203132013B0
:100A5000051A2017A01A2E2DA301A30A201B322D40
:100A6000A401A40AA01D362D0230A307201E3E2B90
:100A70000230A4073E2B8301C5004408BE00BF011D
:100A8000BF00BE014508BE04BF1F562D20143F08FD
:100A9000F1003E08F000F009F10901307007BE00D6
:100AA0000030031801307107BF00572D20100530AA
:100AB000F200F3013F08F1003E08F00095237408AE
:100AC000B2007508B300330DB30CB20C330DB30C88
:100AD000B20C330DB30CB20CA601A501A70132086C
:100AE000BC003308BD003D08803AF0008030700241
:100AF0000A3003193C02031CA82DF6303C073D08C0
:100B000003183D0AFF3E8039031D8B2DA70AF630DE
:100B1000BC07031CBD032708F000F101F63E710875
:100B20000318710AFF3E8039031D992DA50AF6307E
:100B3000A7072508F000F101F63E71080318710AB5
:100B4000FF3E8039031D732DA60AF630A507732DCD
:100B50003C08BA003D08BB002708B800B9012508C9
:100B6000B600B7012608B400B501201CBA2D0B3021
:100B7000B400B501A608031D0800A508031DEC2D4F
:100B8000A708031DE12D3D083C04031DD42D0A30A8
:100B9000B800B901B6003908B7003608B400370804
:100BA000B500BA01BB010800201CD82D0B30D92D8F
:100BB0000A30B600B7010A30B400B501B801B90176
:100BC0000800201CE52D0B30E62D0A30B600B701D9
:100BD0000A30B400B5010800201CF22D0B30B4001F
:100BE000B50108000A30B400B50108006400DD2436
:100BF000FD23803083169F008312B1012112A111C1
:100C00000030211A0130AC000030A1190130AC00D5
:100C10000030211A0130AC000030A2180130AC00C5
:100C20000030A11A0130AC000030211B0130AC00B3
:100C30003E231F1F232E21162A2E1F1B2A2E83160A
:100C40009F0A8312B10A3E23640010303102031C54
:100C50001D2EA115211AA42EA119962E0730F100E0
:100C60003108083E7023AC006400A501A701BC0058
:100C7000BD013D08803AF000803070020A3003194F
:100C80003C02031C612E6400F6303C073D0803184B
:100C90003D0AFF3E8039031D522EA70AF630BC07DD
:100CA000031CBD032708F000F101F63E710803188C
:100CB000710AFF3E8039031D392EA50AF630A707B9
:100CC000392E3C08B8003D08B9002708B600B70126
:100CD0002508B400B501A218742E0830310203189B
:100CE000732EA1162117A214A11ABA2E0530C60020
:100CF000003066237C233C30B824C330B824350848
:100D000034040319882E0530F10034087023892E2D
:100D10003230B8240530F10036087023B8243C3056
:100D2000B8240530F10038087023B42E0530C60011
:100D3000003066237C235E23BE30B8240530B824FF
:100D40001E30B824CD30B82EA218A92EA116A21498
:100D50002117A11ABA2E0530C600003066237C2365
:100D60005E23B930B8241E30B824CD30B8243230D8
:100D7000B824BB2E7624C601003066233230B82456
:100D80009130B8249630B8249B30B824A030B824D1
:100D90009630B8247830B8244B30B824A530B82425
:100DA000AA30B8247830B8244B30B8243230B82474
:100DB0003230B824C601C60A00306623C42302308C
:100DC000C600003066234630B8244B30B82450307B
:100DD000B8245530B8245A30B824AF30B824033082
:100DE000C600003066235F30B8245030B824643029
:100DF000B8246930B8244B30B824AF30B82404305C
:100E0000C60000306623C4238B1306258B172303EB
:100E10000319712F2308023A0319612F8B13CC3069
:100E200055248B17A1181B2F8B13443055248B1777
:100E3000A114AF01A113A118061D252FA11F252F55
:100E40008B13BE3055248B17A0178823A01F832F28
:100E50008B13E023A800E023AA008B17C400280806
:100E60003B25A113A110A0130230C6002A3066232F
:100E70000530F10034087023B8240530F10036083D
:100E80007023B8240530F10038087023B824A60870
:100E9000031D562FA508031D562FA708031D562F07
:100EA0003D083C04031D562F3230572F3C30B824E8
:100EB0000530F1003A087023B8244130B824463098
:100EC000822F0230C6002A3066233230B8246E30BA
:100ED000B8247330B8247830B8247D30B8248230F8
:100EE000802F0230C6002A3066233230B824873083
:100EF000B8243C30B8248C30B8243C30B82432308C
:100F0000B8243230B82424030319ED2F2408023A00
:100F10000319DD2F8B13CC3097248B172119972FB2
:100F20008B13443097248B172115B00122102119FF
:100F3000051EA12F221CA12F8B13BE3097248B17C7
:100F400021148823211CF92D8B131A24A9001A249B
:100F5000AB008B17C40029083B252210211121105A
:100F60000330C6002A3066230530F10034087023B0
:100F7000B8240530F10036087023B8240530F1009C
:100F800038087023B824A608031DD22FA508031D16
:100F9000D22FA708031DD22F3D083C04031DD22FDA
:100FA0003230D32F3C30B8240530F1003A0870239A
:100FB000B8244130B8244630FE2F0330C6002A3012
:100FC00066233230B8246E30B8247330B8247830B9
:100FD000B8247D30B8248230FC2F0330C6002A307C
:100FE00066233230B8248730B8243C30B8248C30A3
:100FF000B8243C30B8243230B8243230B824F92D2B
:02400E003C3F35
:00000001FF
